:100000000C9462000C94CB1A0C94F81A0C948A008D
:100010000C948A000C948A000C948A000C948A0038
:100020000C948A000C948A000C948A000C948A0028
:100030000C948A000C94C2060C948A000C948A00DA
:100040000C94251B0C948A000C94781E0C94B31EFF
:100050000C948A000C948A000C948A000C948A00F8
:100060000C9446050C948A00000000002400270030
:100070002A0000000000250028002B0000000000DE
:1000800023002600290004040404040404040202DA
:100090000202020203030303030301020408102007
:1000A0004080010204081020010204081020000012
:1000B0000007000201000003040600000000000029
:1000C00000005B2011241FBECFEFD8E0DEBFCDBF04
:1000D00012E0A0E0B1E0ECEBF2E402C005900D927A
:1000E000A63BB107D9F714E0A6EBB2E001C01D9220
:1000F000A03AB107E1F710E0C4ECD0E004C02297C9
:10010000FE010E945821C23CD107C9F70E94A020DD
:100110000C945C210C940000FB01DC0102C00190F6
:100120000D9241505040D8F708958091B602813029
:1001300019F482E08093B6028091B602833019F4FC
:1001400084E08093B6020895E3E0F0E089E08093D4
:100150005700849190E08670863009F491E0892FF1
:1001600008951F93182F0E94A400882379F09FB749
:1001700081E08093E603F894A89588E1809360007D
:1001800010936000112309F0A8959FBF1F91089557
:10019000382F20E08091E7039091E803822793278E
:1001A00040E061E270E19C01220F331F97FF04C021
:1001B000C9018627972701C0C9014F5F483099F7C9
:1001C0009093E8038093E70308958436910520F423
:1001D000BC0180E090E025C08E3B910550F48A552B
:1001E0009040BC0180E090E02AE030E040E050E048
:1001F00016C0823D910550F4845B9040BC0180E0C4
:1002000090E024E630E040E050E009C08D5C904092
:10021000BC0180E090E028E532E040E050E00E9440
:10022000AF2024E630E040E050E00E94AF20089587
:1002300090E08C599F4F0E94E5000895DC0198964C
:10024000EC91F0E0E770F070E256FD4F8081089588
:10025000FC0120A530E0C9018170907001962770E3
:10026000307035952795820F931F880F880F08955A
:100270008F929F92AF92BF92CF92DF92EF92FF92B6
:100280000F931F938C010E941E01D80197962C9109
:1002900030E043E150E0249FF001259FF00D349FB2
:1002A000F00D1124E251FE4F80809180A280B38036
:1002B00090E00F96AA2797FDA095BA2FBC01CD011B
:1002C00020E43FE14DE750E00E94AF20A5019401FA
:1002D0000E94E22069017A0180ED97E0A0E0B0E0A1
:1002E000C80ED91EEA1EFB1ED80198968C91887103
:1002F00081F060E07EEE8AEB9BE0A50194010E9414
:10030000E22028513C4F4F4F5F4FC20ED31EE41ED8
:10031000F51E87EE93E0A0E0B0E0C80ED91EEA1EFD
:10032000FB1EC701B60128EE33E040E050E00E941A
:10033000E220CA01B90128EE33E040E050E00E941B
:10034000AF201F910F91FF90EF90DF90CF90BF9063
:10035000AF909F908F9008951F93182FDB01FA01A3
:10036000482F469530E0848190E083709070982FFC
:1003700088272081820F911D11969C938E938481F2
:1003800090E08C70907076E0880F991F7A95E1F775
:100390002181820F911D13969C938E9312978481D5
:1003A00090E08073907064E0880F991F6A95E1F780
:1003B0002281820F911D15969C938E9314978481B0
:1003C00090E0807C9070880F991F880F991F23817F
:1003D000820F911D17969C938E93169735961896BB
:1003E0003F5F431708F0BFCF10FF50C08081829558
:1003F00086958695837090E02DE431E0AC01429FB4
:10040000C001439F900D529F900D11240C961196A0
:100410009C938E93808190E044E0969587954A95D1
:10042000E1F783709070AC01429FC001439F900D33
:10043000529F900D11240C9613969C938E931297B5
:10044000808190E0969587959695879583709070BA
:10045000AC01429FC001439F900D529F900D11240B
:100460000C9615969C938E931497808190E08370E0
:100470009070AC01429FC001439F900D529F900D20
:1004800011240C9617969C938E9316971F9108959E
:1004900023E08032920718F420E030E026C023E009
:1004A000883E920748F49C012F51334054E0369522
:1004B00027955A95E1F719C027E0803D920720F46F
:1004C0009C012C5D334011C028E08839920718F058
:1004D0002FEF33E00AC09C01285C374044E036959A
:1004E00027954A95E1F72D503C4FC90108958C306E
:1004F000910548F49C0174E0220F331F7A95E1F7CF
:10050000285D3C4F17C023E0843F920720F49C01F4
:1005100024523C4F0FC024E08030920718F020E9AD
:1005200038E008C09C012657334F64E0220F331F88
:100530006A95E1F7C90108959C01369527952575BF
:100540003575821B930B9C0136952795369527951B
:100550002373337383739373280F391FC901E4E046
:1005600096958795EA95E1F7820F931F8F709F709C
:1005700021E031E0AC01429FC001439F900D529FAA
:10058000900D1124892F0895882339F02D980000AB
:100590002B9A00002D9A000008952D9800002B98AA
:1005A00000002D9A000008952D9A000083B12D9827
:1005B000000090E0B4E096958795BA95E1F78170D8
:1005C00008950F931F93082F5C9A2D985C9810E064
:1005D000802F80780E94C402000F1F5F1830C1F77F
:1005E0002D981F910F9108958F770E94E102089531
:1005F0000F931F93082F10E0802F80780E94C40271
:10060000000F1F5F1830C1F72D981F910F910895AB
:100610000F931F932D9880E000E0182F110F0E9478
:10062000D402810F0F5F0830C1F71F910F91089519
:100630000E94F4020E9408035C9A08951F93162FEB
:1006400080680E94E102812F0E94F8025C9A1F914B
:1006500008951F931091DB021827E2EDF2E0E80FF6
:10066000F11D89E767850E941E038DE3612F0E94BB
:100670001E0382E4612F0E941E031F91089586E2EB
:100680000E94180308950F931F938BE20E94180392
:10069000082F8CE20E941803282F30E096E0369550
:1006A00027959A95E1F710E0000F111F000F111F19
:1006B000202B312BC9011F910F9108950F931F9388
:1006C0008C018CE1F80164810E941E038DE1F80128
:1006D00065810E941E038EE1F80166810E941E035F
:1006E00080E2F80167810E941E0381E2F8016085C3
:1006F0000E941E0382E2F80161850E941E0383E2CC
:10070000F80162850E941E0384E2F80163850E945D
:100710001E0385E2F80164850E941E038AE2F80147
:1007200065850E941E038EE6F80166850E941E0301
:100730008FE6F80167850E941E0380E7F801608953
:100740000E941E0381E7F80161890E941E0382E76F
:10075000F80162890E941E031F910F910895EF9284
:10076000FF920F931F93CF93DF937B018C01603037
:1007700028E372072CE982072CE1920728F520E88C
:1007800036E948E950E00E94E220E9016897B901A2
:1007900080E090E020E839E647E65FEF0E94AF2076
:1007A0006E0D7F1D801F911F32E0660F771F881F1F
:1007B000991F3A95D1F721E732E040E050E00E94DE
:1007C000E220890180E421C020E03DE241E351E0E4
:1007D0000E94E220E9016897B90180E090E020E002
:1007E00033ED4EEC5EEF0E94AF206E0D7F1D801F3B
:1007F000911F660F771F881F991F21E732E040E0A5
:1008000050E00E94E220890180E69E012F71622F54
:10081000680F85E70E941E0386E7612F0E941E0372
:1008200087E7602F0E941E03CDB7DEB7E6E00C9489
:1008300047219F92AF92BF92CF92DF920F93DF93A7
:10084000CF9300D000D0CDB7DEB7982E83E00E94C2
:1008500018038093FB0284E00E9418038093FC023B
:1008600086E060E00E941E0387E061E00E941E03B4
:1008700089E06FE70E941E038AE065E00E941E0384
:100880008BE062E10E941E038CE065E10E941E0382
:100890008DE06DEF0E941E038EE060E00E941E035B
:1008A000992019F08DE492E008C08091F90223E1CB
:1008B000829FC001112482519E4F0E945E0380E3FB
:1008C0006CE80E941E0382E36FE00E941E0383E334
:1008D00062E40E941E0384E36AE00E941E0385E333
:1008E0006AE20E941E0386E36DE20E941E0387E314
:1008F00064ED0E941E0388E360E00E941E0389E30A
:1009000060E00E941E03992049F065E8A62E61EC84
:10091000B62E61ECC62E6EEDD62E08C0A090DB027E
:10092000B090DC02C090DD02D090DE020AE38D2D93
:100930009927AA27BB2789839A83AB83BC83802FFF
:1009400069810E941E03802F8B5F69810E941E03B4
:10095000DC2CCB2CBA2CAA240F5F0E3341F783E496
:100960006FEF0E941E0384E46FEF0E941E0385E474
:100970006FEF0E941E0386E46FEF0E941E03992012
:1009800019F08DE666E003C08DE66091DF020E94FB
:100990001E0389E760E00E941E038AE76091E0027F
:1009A0000E941E0383E760E00E941E0384E760E06C
:1009B0000E941E03992029F060EC7AEC89E896E306
:1009C00008C06091D7027091D8028091D9029091AD
:1009D000DA020E94AF030F900F900F900F90CF910B
:1009E000DF910F91DF90CF90BF90AF909F900895CF
:1009F00087E061E00E941E038EE764E20E941E030E
:100A000088E063E00E941E0388E060E00E941E030D
:100A100087E065E00E941E0385E062E00E941E03FD
:100A200083E00E9418038093FB0284E00E94180375
:100A30008093FC02089590E0411191E0880F982B7B
:100A40009093BA00660F6093BD0030930203209329
:100A500001030895882311F085EC01C085E8809397
:100A6000BC00089585ED8093BC008091BC0084FD9E
:100A7000FCCF089585EC8093BC000895ECEBF0E08A
:100A8000108285E480831092070308951F920F92CD
:100A90000FB60F9211242F933F934F935F936F9351
:100AA0007F938F939F93AF93BF93EF93FF93DF93C6
:100AB000CF930F92CDB7DEB78091B90090E0887FD9
:100AC00090708036910509F4EAC081369105CCF525
:100AD0008832910509F47CC089329105B4F48031E3
:100AE000910509F470C0813191053CF4009709F437
:100AF0000EC1089709F00DC166C08831910509F44F
:100B000067C0809709F005C177C08034910509F46A
:100B100090C08134910544F48033910509F46EC08E
:100B2000C89709F0F6C06CC08035910509F471C012
:100B30008835910509F483C08834910509F0E9C02E
:100B4000A5C08839910509F4DCC089399105ECF418
:100B50008837910509F4A3C0893791054CF488368C
:100B6000910509F49CC08037910509F0D2C097C067
:100B70008838910509F4C5C08039910509F492C0FF
:100B80008038910509F0C5C08DC0803B910509F4FE
:100B9000A5C0813B91054CF4803A910509F499C0B8
:100BA000883A910509F0B5C099C0803C910509F4D7
:100BB000AAC0883C910509F4A6C0883B910509F0BC
:100BC000A8C080E08CC0809103038093BB009BC0D1
:100BD000809106038150809306038F5F09F43FC024
:100BE000E0910403F091050381918093BB00F093A1
:100BF0000503E093040387C082E049C083E047C057
:100C000084E080930803809107038B7F8093070320
:100C100062C08091BB00E0910403F09105038193D1
:100C2000F0930503E09304038091060381508093C1
:100C3000060380910603823008F065C062C080918F
:100C4000BB00E0910403F09105038193F093050349
:100C5000E093040380910603815080930603809102
:100C600007038B7F809307038091070380FF4FC0AA
:100C7000809107038E7F8093070380910703826032
:100C80008093070384EA8093BC0043C085E080938F
:100C90000803809107038B7F8093070338C010926D
:100CA000060331C0E0910103F0910203309749F14E
:100CB0009091BB00809106038F5F80930603815063
:100CC00011F060E001C062E09983CE0101960995C0
:100CD0001BC00E9432050E943A051BC081E0E091D2
:100CE0000103F0910203309761F0882311F461E071
:100CF00001C063E0CE010196099599819093BB00F4
:100D000003C080E001C081E00E942A0502C00E9469
:100D100032050F90CF91DF91FF91EF91BF91AF918D
:100D20009F918F917F916F915F914F913F912F9103
:100D30000F900FBE0F901F90189525B190E0FC0109
:100D4000EE0FFF1FE80FF91FE259FC4F8081282B9F
:100D500025B988B19181892B88B98BB19281892B72
:100D60008BB9089585B190919E03892385B988B187
:100D700090919F03892388B98BB19091A003892317
:100D80008BB908951F920F920FB60F9211241F93E3
:100D90002F933F934F935F936F937F938F939F9383
:100DA000AF93BF93CF93DF93EF93FF9310914103E2
:100DB00080918402C0918202D0918302181708F0BA
:100DC0005BC08091A1039091A203909387008093D0
:100DD0008600E12FF0E0EE0FFF1FE05AFD4F80810B
:100DE00091810E947702880F991F9093A2038093AC
:100DF000A1038091A1039091A2039E01281B390BAE
:100E0000C90130938302209382022091CD02309158
:100E1000CE02220F331F8217930720F430938302F0
:100E20002093820280914303882339F48091C50284
:100E300080FF59C0183008F456C08FEF9FEF909391
:100E4000890080938800809184009091850080972C
:100E5000D0F30E94B20680914203882339F4809136
:100E60004103882319F081500E949D06809141031F
:100E70008F5F809341033EC08091A1039091A203B4
:100E80009093870080938600D093A203C093A10320
:100E900080914303882319F08FEF9FEF06C0809164
:100EA000A1039091A203885592409093890080936A
:100EB000880080E49CE99093830280938202809171
:100EC0008400909185008097D0F30E94B2068091B3
:100ED0004203882329F48091840281500E949D0658
:100EE0001092410307C08091A1039091A2038855FD
:100EF0009240A5CFFF91EF91DF91CF91BF91AF913C
:100F00009F918F917F916F915F914F913F912F9121
:100F10001F910F900FBE0F901F90189590E0880FB3
:100F2000991F880F991F8C30910518F42CE030E040
:100F300007C09C0183E0253F380710F024EF33E021
:100F4000C90108950F931F930091C6020033C0F4A6
:100F5000202F30E0C90180739070009719F04097FE
:100F600049F403C080913B0307C080914003829500
:100F7000807F02C080913A0389010F70107016C003
:100F80000F33E8F410E00F701070809140038295E9
:100F9000807F0E948E07F801EE0FFF1FE05AFD4F81
:100FA000918380830F5F1F4F80913A030E948E07C9
:100FB000000F111F005A1D4FF801918380831F916C
:100FC0000F9108951F9380914503909146038F5F81
:100FD0009F4F39F11091C602412F50E04F70507071
:100FE000BA016F5F7F4FA5E4B3E020E030E0241743
:100FF000350789F02617370711F4103360F4F89499
:101000008D919C911197F901EE0FFF1FE05AFD4F52
:101010009183808378942F5F3F4F12962031310562
:1010200031F71F910895982F8091BA02873269F4A1
:10103000992331F08091B00080618093B0000895D1
:101040008091B0008F7E8093B00008951F93CF935E
:10105000DF93EC0170E0CB018270907060FF1AC0EA
:10106000892B31F08091670388831092E50345C096
:101070001091E50382ED92E00E941E011817D8F549
:10108000E12FF0E0ED55FC4F808188831F5F1093C6
:10109000E50333C0892BC1F098819093E40310924B
:1010A000E503892F807E803651F48091670382307A
:1010B00010F188818F718093250383E01AC09E3FD1
:1010C000E1F41092670317C08091E4038F3FA9F405
:1010D0002091E503293278F4E22FF0E0EE52FD4F43
:1010E00088818083822F8F5F8093E503893229F482
:1010F00081E08093670380E001C081E0DF91CF91C0
:101100001F910895EF92FF920F931F93CF93DF9358
:1011100080E260E040E026E238E00E941B05109289
:10112000670392E0E92E85E0F82E04E080916703E2
:10113000813039F480E00E941904E09267034398FB
:10114000F5CF10916703133061F442988091250325
:101150000E9429031093B6020E94F80400936703CB
:10116000E5CF80916703843009F78091B60284301F
:10117000E9F68FE70E94F402C0E0D0E007C00E94C9
:101180000803FE01ED55FC4F8083219682ED92E02D
:101190000E941E0190E0C817D9078CF3F0926703F4
:1011A000429AC4CFA0E0B0E0E8EDF8E00C9427212B
:1011B000EC010E947B1B5B016C017E0100E010E0F2
:1011C00011C0209779F00E947B1B6A197B098C095A
:1011D0009D09E616F7060807190720F40E943E0548
:1011E00081E008C08091070382FDEBCF8091080366
:1011F00010920803CDB7DEB7EAE00C944321A0E0DB
:10120000B0E0E5E0F9E00C942921182F7B01042FD0
:10121000C22FD0E024E0C22ED12CCC22DD22C2FF8E
:1012200003C080E090E004C0809180029091810230
:101230000E94D208282F8823B9F510920803009342
:101240000603F0920503E0920403110F116010935E
:10125000030390910703C1FD02C084E001C085E053
:10126000892B809307038091070381FF0BC0809136
:1012700007038D7F80930703809103038093BB0056
:1012800085EC01C085EE8093BC00C0FF0DC0C11489
:10129000D10419F080E090E004C080918002909128
:1012A00081020E94D208282F822FCDB7DEB7E8E056
:1012B0000C944521A0E0B0E0E0E6F9E00C9429218F
:1012C000182F7B01042FC22FD0E034E0C32ED12C85
:1012D000CC22DD2222FF03C080E090E004C0809198
:1012E0008002909181020E94D208282F8823B1F5B4
:1012F0001092080300930603F0920503E0920403A2
:10130000110F1093030390910703C1FD02C084E005
:1013100001C085E0892B809307038091070381FF3B
:101320000BC0809107038D7F809307038091030397
:101330008093BB0085EC01C085EE8093BC00C0FFAC
:101340000DC0C114D10419F080E090E004C0809178
:101350008002909181020E94D208282F822FCDB75F
:10136000DEB7E8E00C9445218091B602813011F09F
:1013700081E008950E947B1B2091FD023091FE02C6
:101380004091FF0250910003621B730B840B950B7D
:10139000615A76488140904010F480E0089582E0E0
:1013A0000895FF920F931F93CF93DF93182F092F68
:1013B000F62E8EE30E941E03212F302FC901EC016F
:1013C00010E005C08FE769910E941E031F5F1F1583
:1013D000C8F385E064E00E941E0383E00E941803C6
:1013E0008093FB0284E00E9418038093FC020E9419
:1013F0007B1B6093FD027093FE028093FF0290932B
:10140000000387E069E00E941E0381E08093B6023A
:10141000CDB7DEB7E5E00C9448210E94D109809158
:10142000B6028130D9F40E947B1B2091FD023091DD
:10143000FE024091FF0250910003621B730B840B6C
:10144000950B605A76488140904040F4E8CF8EE793
:1014500094E060E071E00E94631E08958091B602FE
:101460008130A9F30895A1E0B0E0E9E3FAE00C943B
:101470002F21809167038230B9F480E2BE016F5F53
:101480007F4F41E021E00E94FF08882379F08FEF31
:10149000809367030E946D1B6093680370936903D8
:1014A00080936A0390936B038FEF01C0898121962B
:1014B000E2E00C944B21A1E0B0E0E1E6FAE00C940C
:1014C0002F21809167038230D9F480912503805ABF
:1014D000898380E2BE016F5F7F4F41E021E00E947F
:1014E0005A09882369F08FEF809367030E946D1B70
:1014F000609368037093690380936A0390936B030E
:101500002196E2E00C944B21AAE2B0E0EAE8FAE08E
:101510000C942D218FEF8983DE011296E2EDF2E02B
:1015200089E201900D928150E1F780E28E010F5F18
:101530001F4FB8014AE221E00E945A09882351F462
:1015400080E2B80141E021E00E94FF08882311F405
:1015500082E001C08FEF8093670380916703823040
:1015600051F00E946D1B6093680370936903809330
:101570006A0390936B03AA96E4E00C944921A2E0DD
:10158000B0E0E5ECFAE00C942B210E947B1B9B0160
:10159000AC018091090390910A03A0910B03B091D3
:1015A0000C0379018A01E81AF90A0A0B1B0BD8010E
:1015B000C70181519742A040B04008F444C08091D7
:1015C0000D038F5F80930D03815080FD02C000E00A
:1015D00001C007E02093090330930A0340930B03F3
:1015E00050930C038EE794E063E00E941B208EE78B
:1015F00094E061E00E941B2077E0F72EF00E802F30
:1016000090E0880F991F9C01205A3D4F3A8329830F
:10161000F90160817181672F772763707070880F7F
:10162000991F682B792B8EE794E00E941B20E9819B
:10163000FA816081718170708EE794E00E941B20B6
:101640000F5F0F15E1F62296E6E00C9447211F93F9
:10165000182F8EE794E0612F0E941B20812F0E949B
:10166000C8001F910895A0E0B0E0E9E3FBE00C940E
:101670002921082F0E947B1B9B01AC01809109034B
:1016800090910A03A0910B03B0910C0369017A01B8
:10169000C81AD90AEA0AFB0AD701C6018151974242
:1016A000A040B04008F443C02093090330930A03DC
:1016B00040930B0350930C031092E8031092E7033E
:1016C00088EA0E94270B002311F481E001C081E821
:1016D0000E94270B80E10E94270BC0E0D0E0FE01B2
:1016E000EE0FFF1FE05AFD4F808191810E9477022B
:1016F0008C01E3E0000F111FEA95E1F7812F0E94B2
:10170000270B802F0E94270B2196C031D10539F776
:101710006091E8038EE794E00E941B206091E7034C
:101720007091E80370708EE794E00E941B20CDB7A3
:10173000DEB7E8E00C944521A0E0B0E0E2EAFBE08F
:101740000C942921182F062F0E947B1B9B01AC01B2
:101750008091090390910A03A0910B03B0910C03AF
:1017600069017A01C81AD90AEA0AFB0AD701C60137
:1017700081519742A040B04008F4D6C1209309039C
:1017800030930A0340930B0350930C038091600243
:1017900090916102880F991F80930E03977080913A
:1017A0000F03887F892B80930F0320916202309171
:1017B0006302220F331F922F990F990F990F877091
:1017C000892B80930F03422F429546954770809155
:1017D0001003807C932F9770990F990F990F842B8A
:1017E000892B809310032091640230916502220FAF
:1017F000331F922F9295990F990F907C8F73892B9D
:1018000080931003932F9295990F990F907C822FBC
:1018100086958695892B80931103932F969596959F
:101820009170809112038E7F892B809312032091F7
:10183000660230916702220F331F922F990F817039
:10184000892B80931203422F441F4427441F809109
:101850001303807F932F9770990F842B892B80938C
:1018600013032091680230916902220F331F922FD7
:101870009295907F8F70892B80931303422F42950E
:101880004F70809114038078932F97709295907F7A
:10189000842B892B8093140320916A0230916B0270
:1018A000220F331F8F7780931403932F97959927D7
:1018B0009795822F8695892B80931503932F969564
:1018C0009370809116038C7F892B8093160340912F
:1018D0006C0250916D02440F551F942F990F990F70
:1018E0008370892B80931603942F929596959695E5
:1018F000937020911703207E852F8770880F880FA3
:10190000292B282B2093170380916E0290916F0250
:10191000880F991F382F3295330F307E2F71232B6C
:1019200020931703292F2295220F207E86958695D6
:101930008695822B8093180380917002909171029A
:10194000880F991F80931903977080911A03887FDD
:10195000892B80931A032091720230917302220F17
:10196000331F922F990F990F990F8770892B8093AE
:101970001A03422F42954695477080911B03807C45
:10198000932F9770990F990F990F842B892B809320
:101990001B032091740230917502220F331F922F86
:1019A0009295990F990F907C8F73892B80931B03CD
:1019B000932F9295990F990F907C822F86958695FB
:1019C000892B80931C03932F969596959170809107
:1019D0001D038E7F892B80931D0320917602309109
:1019E0007702220F331F922F990F8170892B8093DA
:1019F0001D03422F441F4427441F80911E03807FF4
:101A0000932F9770990F842B892B80931E0320911D
:101A1000780230917902220F331F922F9295907F96
:101A20008F70892B80931E03422F42954F708091B7
:101A30001F038078932F97709295907F842B892B2A
:101A400080931F0320917A0230917B02220F331F73
:101A50008F7780931F03932F979599279795822FC0
:101A60008695892B80932003932F96959370809170
:101A700021038C7F892B8093210340917C0250911C
:101A80007D02440F551F942F990F990F8370892B56
:101A900080932103942F929596959695937020911B
:101AA0002203207E852F8770880F880F292B282BF3
:101AB0002093220380917E0290917F02880F991FCC
:101AC000382F3295330F307E2F71232B2093220332
:101AD000292F2295220F207E869586958695822B2A
:101AE00080932303112311F490E001C098E00023B8
:101AF00011F480E001C084E0892B809324038EE7F9
:101B000094E06FE00E941B20CEE0D3E08EE794E0EB
:101B100069910E941B2083E0C532D807B9F78EE790
:101B200094E060E00E941B20CDB7DEB7E8E00C94A3
:101B3000452180913E0390913F039F770E949C0234
:101B4000982F809340038F3029F480913A03869533
:101B5000805804C089E0989FC001112480933B0302
:101B6000F8940E94A20778948091BA028132C9F455
:101B700090913B03892F81508E3F60F08091B0009F
:101B80008F7D8093B00060E0911161E083E00E945E
:101B9000761C08959093B4008091B0008062809389
:101BA000B00008951F93182F811111E082E1612F79
:101BB0000E94761C83E1612F0E94761C109206031E
:101BC000109207038091B9008C6F8093B90080E276
:101BD0008093B80085E48093BC001F910895CF9353
:101BE000DF938EE794E00E94A81F892BF9F0809183
:101BF000E203C82FD0E09E012F5F3F4F2F7130705E
:101C00008091E10390E02817390781F08EE794E096
:101C10000E94E21FCF53DC4F88838091E20390E063
:101C200001968F7190708093E203DBCFDF91CF91AB
:101C30000895EF92FF921F93CF93DF9382ED92E08E
:101C40000E942801482F809384025091C602252FBC
:101C500030E02F70307090E02817390719F44F5F8B
:101C60004093840250535F3058F440918402842F93
:101C700090E001972817390719F44F5F40938402C9
:101C800080918402813118F080E180938402EEE635
:101C9000F3E0108211821282339623E0E038F207DB
:101CA000C1F78FEF80939E0380939F038093A003DF
:101CB00088EBE82E82E0F82EACE8B2E0E7016FEFA7
:101CC0005FEF4FEF88818031F0F490E03C91FC01B0
:101CD000EE0FFF1FE80FF91FE259FC4F8081832BA5
:101CE000808311962C9111978181822B818312968A
:101CF0009C9112978281892B828330954323209572
:101D00005223909569232196139682E0CE3BD80703
:101D1000C9F66093A00350939F0340939E03C6E8C7
:101D2000D2E010E0F7018081823238F08632B0F0E4
:101D3000863219F4888160E00FC0143021F480915C
:101D4000C1008F7E05C0153029F48091C100877FC6
:101D50008093C100888161E00E940A1C1F5F089483
:101D6000E11CF11C21961630E9F68091B802803210
:101D700031F489E061E00E94761C82E801C082E0D3
:101D80008093800081E0809342038093430380919D
:101D9000BA02813211F08732D9F483E061E00E9407
:101DA0000A1C83E060E00E94761C8091BA028132B6
:101DB00031F481E08093B0008093B10009C082E0EB
:101DC0008093B00085E08093B1008EE38093B300F0
:101DD0008AE1809381008FEF9FEF90938900809339
:101DE000880080ED97E0909387008093860080E4E0
:101DF0009CE990938302809382029093A203809344
:101E0000A1031092410380916F00816080936F0065
:101E10008091C50283FF0DC08091450390914603D8
:101E20008F5F9F4F31F00E94E207109243031092A0
:101E30004203DF91CF911F91FF90EF9008958CE0C6
:101E400060E00E940A1C8BE061E00E940A1C8DE0A9
:101E500061E00E940A1C82E060E00E940A1C84E0AB
:101E600061E00E940A1C089583E00E941803809399
:101E7000FB0284E00E9418038093FC0287E061E08B
:101E80000E941E036AE070E080E090E00E94A11BC7
:101E90000E94F804000008950F931F93082F17C0A5
:101EA000439A64E670E080E090E00E94A11B4398B2
:101EB00064E670E080E090E00E94A11B1F5F1017B5
:101EC00078F36CE271E080E090E00E94A11B10E0EA
:101ED000F6CF482F392F25E00DC0F999FECF1FBA54
:101EE000842F932F92BD81BD60BD0FB6F894FA9AEE
:101EF000F99A0FBE215059F0F999FECF842F932FF4
:101F000092BD81BDF89A80B5681739F7089582E0CF
:101F10000E944C0F0895A0E0B0E0E1E9FFE00C94CE
:101F20002121482E562EEE24FF24C0E0D0E0CC2400
:101F3000DD248824992404C055245394CC24DD2422
:101F4000442051F467EBE62E62E0F62EC0E0D0E0CC
:101F50005BE1852E912C19C021E0421651F442ED2F
:101F6000E42E42E0F42ECDE1D0E039E2832E912C34
:101F70000CC032E0431649F425E4E22E23E0F22EB1
:101F8000C8E4D0E090E2892E912C3E016C0C7D1CBF
:101F90001092E8031092E703E3011BC0552059F4A7
:101FA000F999FECFD2BDC1BDF89A80B5F701E00F17
:101FB000F11F808307C0F701E00FF11FCE016081A0
:101FC0000E94690F0E0D1F1DF80180810E94C8003C
:101FD00021969E012619022F10E008151905F0F22E
:101FE000CE015520D9F4F999FECFD2BDC1BDF89AE2
:101FF00020B5F999FECF2196D2BDC1BD2197F89A9F
:1020000080B590E0B22EAA248A299B292091E7036B
:102010003091E8032817390759F48ECF2196609143
:10202000E8030E94690FCE016091E7030E94690FE7
:1020300080E091E0C80ED91E91E0C91693E0D90660
:1020400008F47ECF852DCDB7DEB7E0E10C943D21BD
:1020500082E060E00E948B0F882331F48FEF9FEFC6
:102060009093460380934503089582E061E00E94C7
:102070008B0F089596E09093B70290E29093B80288
:1020800026E22093B90291E29093BA022093BB0218
:1020900094E29093BC0295E29093BD0292E09093FB
:1020A000C5029FEF9093C6022AE02093CF021092C0
:1020B000D0021092D1021092C7021092C802109260
:1020C000C9021092CA029EE19093CB022093CC02E7
:1020D00028EB3BE03093CE022093CD02882361F0C1
:1020E00080E061E00E948B0F8FEF9FEF909346039B
:1020F000809345030E9435100895ABE5B0E0E3E816
:10210000F0E10C941F215B016C010E946D1B1B010F
:102110002C0181E00E94190483E08093B6020E94A2
:10212000340F8EE794E06CE071E00E94631E3E0184
:102130000894611C711CE4C08EE794E06AE171E0D0
:102140000E94631E8FE70E94F4020E940803182F6A
:102150008983823601F502ED12E00E940803F8013E
:1021600081938F01F2E00B3F1F07B9F78091D202F4
:10217000873309F0C0C08EE794E063E271E00E940B
:10218000631E82E48983CE01019661E00E940D0AFC
:10219000429A81E0CBC0803719F0893631F506C00C
:1021A00020E52A83AA24BB24650105C081E00E94A2
:1021B0003A1089E48A838091E603882321F0809194
:1021C000C502806803C08091C5028F778093C502E5
:1021D000DE011396E7EBF2E08BE101900D92815066
:1021E000E1F7CE0102966CE184C08437E1F434E576
:1021F0003E8F83E08F8F93E798A3E6E0E9A3FCE0AE
:10220000FAA3DE019396E6EDF1E088E101900D92EC
:102210008150E1F7CE014E966DE10E940D0AAA248D
:10222000BB24650168C0853791F407EB12E00E947A
:102230000803F80181938F01F2E0023D1F07B9F70F
:1022400080E061E00E948B0F25E5298350C086362F
:1022500031F580914503909146038F5F9F4FD1F0F8
:1022600086E48BAF75E4E72E73E0F72E8E01045CF5
:102270001F4FF701819191917F010E947702F80130
:10228000908381830E5F1F4FF5E6EF16F3E0FF06A4
:1022900081F701C01BAFCE01CB9661E22AC0873621
:1022A000D9F405E413E00E940803982E88240E94C4
:1022B00008039401280F311DC9010E944802F8014A
:1022C000819391938F01F3E005361F0761F727E4AF
:1022D00029830E9435100BC0873469F48FEF9FEF7C
:1022E00090934603809345030E9435101983C301E0
:1022F00061E00E940D0A93E09093B6020E94F804F8
:10230000A114B104C104D10459F00E946D1B6219DB
:102310007309840995096A157B058C059D0528F4C8
:102320008091B602843061F707CF80E0C55ADF4F55
:10233000E2E10C943B2180E060E00E948B0F882357
:1023400019F481E00E943A10089581E061E00E9452
:102350008B0F089581E060E00E948B0F882311F4B9
:1023600090E006C090E08091D202873309F491E0BA
:10237000892F0895EF92FF920F931F93CF93DF93CE
:10238000EB019C01442737FD4095542F60E271EA30
:1023900087E090E00E94042189011216130614F0D0
:1023A00001E010E0BE01882777FD8095982F20E29C
:1023B00031EA47E050E00E94AF209801442737FD02
:1023C0004095542F0E9404217901C0E0D0E009C05B
:1023D0002B9AC8010E94C51B2B98C8010E94C51BDF
:1023E0002196CE15DF05A4F3CDB7DEB7E6E00C9459
:1023F00047211F93182F429A83E00E94180380936D
:10240000FB0284E00E9418038093FC0286E060E0F7
:102410000E941E0387E061E00E941E0389E06FE7CF
:102420000E941E038AE065E00E941E038BE062E1C9
:102430000E941E038CE065E10E941E038DE06DEF9B
:102440000E941E038EE060E00E941E0380E76CE2A3
:102450000E941E0380E360E00E941E0389E760E0A3
:102460000E941E038AE765E00E941E0381E762E185
:102470000E941E0382E762E00E941E0383E760E081
:102480000E941E0384E760E00E941E036091C70261
:102490007091C8028091C9029091CA020E94AF0354
:1024A0008DE667E00E941E036AE070E080E090E045
:1024B0000E94A11B87E069E00E941E036AE070E0B1
:1024C00080E090E00E94A11B112369F010E007C09A
:1024D00088EB91E061E070E00E94BA11A8951F5F5F
:1024E0001531B1F74BC088E891E061E070E00E94DF
:1024F000BA11A8958DE665E00E941E036AE070E0BF
:1025000080E090E00E94A11B88EB91E061E070E028
:102510000E94BA11A8958DE664E00E941E036AE04D
:1025200070E080E090E00E94A11B8DE591E061E009
:1025300070E00E94BA11A8958DE662E00E941E0329
:102540006AE070E080E090E00E94A11B8FEA90E0DA
:1025500061E070E00E94BA11A8958DE660E00E94EB
:102560001E036AE070E080E090E00E94A11B85E01D
:1025700091E062E070E00E94BA11A89587E061E006
:102580000E941E0342981F910895A6E1B0E0EBEC73
:10259000F2E10C942121A8958CE00E941803882375
:1025A00059F48EE794E06EE271E00E94631E80E0D1
:1025B0000E9419040E94340F0E94EF0D0E947B1BA1
:1025C0000E94330A90E0853009F491E08E010F5F9C
:1025D0001F4FBB24BA948091B602843019F099231E
:1025E00009F488C10E947B1B6B017C018091B602BB
:1025F0008430F1F48FE70E94F40200E010E008C09C
:102600000E940803F801ED55FC4F80830F5F1F4FB8
:1026100082ED92E00E941E0190E00817190784F3F2
:102620000E94430390933D0380933C03429A29C048
:1026300082ED92E00E941E01482F4F5F80E2B801B8
:1026400021E00E94FF08882371F0B09267030E9486
:102650006D1B609368037093690380936A03909382
:102660006B0390E0B8CF82ED92E00E941E01482FEC
:1026700023EA33E0FE013296C901BF0150E00E9417
:102680008C00C0922603D0922703E0922803F09298
:1026900029031092660380913E0390913F03880FB7
:1026A000991F816090933F0380933E03439880E09D
:1026B0000E9413088091A303282F30E0C9018E7374
:1026C0009070892B99F5F8948091FA02877060E6F2
:1026D00072E044EA53E00E94AC010E94A2077894A1
:1026E0008091A30390916D0380FF1BC0992309F093
:1026F00045C0A5E4B3E020E030E0F901EE0FFF1F94
:10270000E05AFD4F808191818D939D932F5F3F4FC4
:102710002031310591F70E94351081E080936D03DF
:102720002DC0992359F110926D0328C0C9018873F7
:102730009070C89719F54091B803842F822787FFBE
:102740001DC040584093B8038091BD028532B1F45A
:1027500010E00AC01F5FE12FF0E0ED55FC4F8EE75F
:1027600094E060810E941B20212F30E08091A30320
:1027700090E0877090708217930764F780916503EB
:10278000882319F481E0809365031092440310922A
:102790004203109243038091FA02887109F4A1C0A8
:1027A0004091B8038091A30390E0242F30E082276A
:1027B000932786FD60C0407C80E448274093B8039F
:1027C0009091E1038091E203981701F1A9EBB3E046
:1027D00030E00FC03F5F892F90E0FC01EF53FC4FCA
:1027E00020812D9301968F7190708093E103383092
:1027F00031F09091E1038091E203981759F7395C29
:102800008091B803382B3093B80335C080913903D9
:102810008093B9038091B902863251F482E10E941B
:10282000D91C95958795959587958093BA0302C095
:102830001092BA038091BB02863251F483E10E9468
:10284000D91C95958795959587958093BB0302C074
:102850001092BB0380913D038093BC0380913C03A5
:102860008093BD0380913E0390913F039F770E9428
:102870009C028093BE0388EB93E069E00E94D1093B
:1028800002C00E94EF0D0E94B4098823D1F308EB27
:1028900012E086E8E82E82E0F82EF8018081E82F29
:1028A000F0E0CF01807F9070409791F4EF70F0706E
:1028B000EE0FFF1FE05AFD4F8081918160E08F3F56
:1028C000910511F008F061E0F70180810E94761C0B
:1028D0000F5F1F4F0894E11CF11CF2E00E3B1F0735
:1028E000E1F683E08093B6020E94F80481E08093D1
:1028F0006C0342980E947B1B5B016C010E946D1B64
:102900002B013C0180916603823008F065C0E090A5
:102910002603F0902703009128031091290380914A
:102920002A0390912B03A0912C03B0912D038E15B7
:102930009F05A007B10709F44FC082ED92E00E9405
:102940003801A60195012E193F09400B510B6C5D12
:102950007540804090406217730784079507E0F543
:10296000E0922A03F0922B0300932C0310932D0383
:102970000E943F038093390320913703309138033D
:10298000280F311D309338032093370360913603AD
:102990006F5F609336036930F8F0C90170E00E9400
:1029A000CE20CB01709338036093370320913A0314
:1029B00043E0249F90011124820F931F96958795E1
:1029C0009695879580933A030E94990D109238034B
:1029D0001092370310923603809165039090E303C1
:1029E000882309F463C180906603891408F0E1C16B
:1029F00082ED92E00E943801209126033091270356
:102A00004091280350912903A21AB30AC40AD50A97
:102A100068517C4F8F4F9F4F6A157B058C059D0534
:102A200008F077C080913E0390913F03880F991F73
:102A300090933F0380933E0381E080936C03882052
:102A400081F440922E0350922F03609230037092D3
:102A50003103109232031092330310923403109218
:102A60003503809166038F5F8093660382ED92E069
:102A70000E943801209126033091270340912803BA
:102A800050912903260F371F481F591F20932603F3
:102A900030932703409328035093290381E08093C8
:102AA0006C03439A0E9413080E94990D32C082ED74
:102AB00092E00E9438019B01AC0180912603909125
:102AC0002703A0912803B091290386017501E81A14
:102AD000F90A0A0B1B0B682D70E080E090E00E9461
:102AE000AF206E157F058007910798F410923F0381
:102AF00010923E0381E080936C0310923A030E948F
:102B0000990DA0922603B0922703C0922803D09279
:102B1000290380916603882309F4F2C09091CF02C3
:102B2000992389F180914403882369F5892F90E0E6
:102B30000E94E50020912E0330912F034091300335
:102B40005091310383017201E21AF30A040B150B51
:102B50006E157F0580079107B0F481E080934403F0
:102B60000E94E2078091CB020E941801640D751D3E
:102B7000861D971D616060933203709333038093C9
:102B80003403909335039091D1029923F1F0809111
:102B900042038823D1F4892F90E00E94E500209120
:102BA0002E0330912F034091300350913103830164
:102BB0007201E21AF30A040B150B6E157F058007EC
:102BC000910718F481E0809342039091D0029923F9
:102BD000F1F0809143038823D1F4892F90E00E9483
:102BE000E50020912E0330912F0340913003509146
:102BF000310383017201E21AF30A040B150B6E15FF
:102C00007F058007910718F481E08093430380914A
:102C1000C7029091C802A091C902B091CA02009760
:102C2000A105B10509F46CC0809132039091330382
:102C3000A0913403B09135030097A105B10509F4C3
:102C40005FC083017201E81AF90A0A0B1B0B17FD1A
:102C500057C06091CC0270E080E090E028EE33E055
:102C600040E050E00E94AF206E157F05800791077D
:102C700008F046C08091C50290E0E4E09695879503
:102C8000EA95E1F781700E94F91180E00E94190431
:102C90000E94F8040E946D1B616060933203709380
:102CA000330380933403909335032AC082ED92E07E
:102CB0000E9438019B01AC0180912603909127036B
:102CC000A0912803B091290386017501E81AF90A39
:102CD0000A0B1B0B692D70E080E090E00E94AF2092
:102CE0006E157F058007910758F4A0922603B092D5
:102CF0002703C0922803D092290381E080936C03BC
:102D0000809143038823B1F48091BD02883219F485
:102D10000E94BF0A0FC0893239F480914403609148
:102D200066030E949C0B06C08A3221F48091440302
:102D30000E94330B80916C038823B9F0E091250346
:102D4000EF5FE0932503E83131F0F0E0EE52FD4F04
:102D50008785882311F410922503809125030E9412
:102D600029030E945B0A10926C03809167038F3FD6
:102D700021F50E946D1B20916803309169034091F9
:102D80006A0350916B03621B730B840B950B695E96
:102D900073408040904088F00E946D1B60936803F0
:102DA0007093690380936A0390936B030E94840A73
:102DB00004C0891409F0ADCE7ACE6696E0E10C9499
:102DC0003D21FF920F931F93082FF62E61E00E9482
:102DD0000A1C802F61E00E94761C8F2D61E00E940A
:102DE000761C8AE090E00E94C51B8F2D0E94A91CD2
:102DF000892B11F410E00FC0802F60E00E94761C38
:102E00008AE090E00E94C51B8F2D0E94A91C10E053
:102E1000892B09F411E0802F60E00E940A1C802FAA
:102E200060E00E94761C8F2D60E00E94761C812F4E
:102E30001F910F91FF900895EF92FF920F931F93B0
:102E40007C010EE714E0C8016F2D70E04AE050E00D
:102E50000E94E01DC8016EE20E941F1DB701E4E060
:102E600076956795EA95E1F76F707070C8014AE052
:102E700050E00E94E01DC8016EE20E941F1D8FE01D
:102E8000E822FF24C801B7014AE050E00E94E01D9B
:102E90001F910F91FF90EF900895A2E2B0E0E3E55B
:102EA000F7E10C941F218E010F5F1F4F80E1D801C5
:102EB0001D928A95E9F78EE794E066E371E00E943F
:102EC000631E0E94340F20EC3DE948E555E32F8F47
:102ED00038A349A35AA380EC97EFAAEBB7E38B8FF3
:102EE0009C8FAD8FBE8F24EF31E040E050E02F8B00
:102EF000388F498F5A8F80E5C82E83ECD82EE12C6D
:102F0000F12CB0EC4B2EBDE95B2EB8E56B2EB5E392
:102F10007B2E88249924540133241E8A1D8A198A01
:102F20001A8A1B8A1C8AFFC08EE794E00E94E21F67
:102F30008434B9F0853430F48332B9F18C3209F03D
:102F4000CCC044C0833509F0C8C02F8D38A149A139
:102F50005AA1C901DA012C013D01882499245401A8
:102F6000E2C08EE794E064E40E941F1D8EE794E0C7
:102F700040EC5DE968E575E32AE030E00E94031E5D
:102F80008EE794E06CE20E941F1D8EE794E040EC17
:102F900057EF6AEB77E32AE030E00E94031E8EE7EA
:102FA00094E06CE20E943D1DBEC019821A821B8211
:102FB0001C821D821E821F82188619861A861B8615
:102FC0001C861D861E861F86188A3AC0339434E0FC
:102FD000331609F0A8C069817A818B819C8128EE23
:102FE00033E040E050E00E94AF206F8F78A389A3C8
:102FF0009AA36D817E818F8198850E94AF206B8F0F
:103000007C8F8D8F9E8F89859A85AB85BC858F8BB4
:10301000988FA98FBA8F6D857E858F8598890E943C
:10302000AF206B017C0190E2C9169EE4D90690E0C6
:10303000E90690E0F90630F48CE162E30E941E0399
:10304000332471C0A0E3CA16A5E7DA06A0E0EA06B9
:10305000A0E0FA0618F48CE162E2F0CFB0E4CB16FF
:10306000BCE9DB06B0E0EB06B0E0FB0618F48CE14F
:1030700066E2E4CFE0E5CE16E3ECDE06E0E0EE0645
:10308000E0E0FE0618F48CE162E1D8CFF0E6CF165E
:10309000FAEEDF06F0E0EF06F0E0FF0618F48CE150
:1030A00065E1CCCF20E7C21621E1D20621E0E2069D
:1030B00020E0F20618F48CE161E0C0CF30EAC316DC
:1030C00036E8D30631E0E30630E0F30618F48CE18D
:1030D00063E0B4CF8CE165E0B1CFA0ED2A2E280EDD
:1030E00049E0421500F1032D10E0000F111F000F01
:1030F000111F81E090E08C0F9D1F080F191FD80150
:103100006D917D918D919C912AE030E040E050E0FE
:103110000E94AF20620D711D811D911DF801608319
:103120007183828393838EE794E00E94A81F892B8A
:1031300009F0FACE81149104A104B10489F4C30109
:10314000B2010E94AF0361E070E080E090E00E9475
:10315000A11BFFEFFE8B1D8A198A1A8A1B8A1C8A03
:103160002F89388D498D5A8D82169306A406B5068F
:10317000E0F40E943F0329893A894B895C89280F32
:10318000311D411D511D298B3A8B4B8B5C8B3D8929
:10319000381708F48D8B4E89841708F48E8B0894A9
:1031A000811C911CA11CB11C56C0C301B20128EEA8
:1031B00033E040E050E00E94E2208EE794E0BA0164
:1031C000A9012AE030E00E94D11D8EE794E06CE274
:1031D0000E941F1D8EE794E06D894AE050E00E9436
:1031E000F11D8EE794E06CE20E941F1D69897A89C7
:1031F0008B899C89A50194010E94E2208EE794E0CE
:10320000BA01A9012AE030E00E94D11D8EE794E0C6
:103210006CE20E941F1D8EE794E06E894AE050E048
:103220000E94F11D8EE794E06CE20E943D1D4C0C63
:103230005D1C6E1C7F1C8B8D9C8DAD8DBE8D841591
:103240009505A605B70520F44F8C58A069A07AA073
:103250008824992454012F8D38A149A15AA1285EB0
:1032600033404040504009F05ECFA296E2E10C941A
:103270003B2180E065E970E042E050E00E94A81A3E
:103280000895A1E0B0E0E7E4F9E10C942F2180E09B
:103290000E94B10080E161E00E940A1C81E161E0CE
:1032A0000E940A1C0E941F0F80E060E00E940A1C1E
:1032B00081E061E00E940A1C8EE794E040E052EC5D
:1032C00061E070E00E94211F0E949B110E94281063
:1032D0008EE794E063E471E00E94601E83E793E070
:1032E0000E941C178EE794E06AE571E00E94601E60
:1032F0008EE794E068E070E04AE050E00E944C1EE7
:103300000E9439197894439A83E063E10E94E116A0
:10331000882329F0439842980E944D17FBCF89E0FB
:1033200062E10E94E116882329F40E94AA118823F1
:1033300009F006C18EE794E062E671E00E94601E2B
:1033400060E070E080E090E00E947D10882349F00A
:103350000E94A5118EE794E06BE971E00E94631E64
:10336000429A0E94190E22C08091BB02833229F03A
:103370008091C5028B7F8093C5028091C50281FF39
:1033800015C082FD13C064EF71E080E090E00E9400
:103390007D10882359F00E94A5118EE794E06BE917
:1033A00071E00E94631E0E94190E429A8091B90238
:1033B000823239F58091BB02833219F581E00E9497
:1033C000D20D8091C50282FF09C08EE794E066EBC2
:1033D00071E00E94631E0E94820813C064E170E0E5
:1033E00080E090E00E94A11B80E2BE016F5F7F4FF2
:1033F00041E021E00E94FF08882319F481E08093D6
:1034000067038EE794E061EC71E00E94601E8FE03C
:103410000E94B10080E00E9419041092250380E010
:103420000E9429031092E30390E0983158F4292F69
:103430002F5FE92FF0E0EE52FD4F8785882311F0D2
:10344000922FF3CF9093E30383E08093B6020E9420
:10345000340F80916703882311F00E94840A8091C1
:10346000BD02883211F08A3239F48EE794E040E0F0
:1034700052EC61E070E02BC0893271F48EE794E089
:1034800040EA56E861E070E00E94211F8091C2008E
:1034900080628093C20022C08091FA0288718031DC
:1034A00069F04091D3025091D4026091D50270919D
:1034B000D6024A3051056105710538F48EE794E073
:1034C00040E855E260E070E002C08EE794E00E94C0
:1034D000211F04C08EE794E00E94E21F8EE794E073
:1034E0000E94A81F892BB1F78091BC02843229F079
:1034F0008091C1008F7E8093C1008091BD02853292
:1035000059F08A3249F0893239F0883229F08091B5
:10351000C100877F8093C1001092E1031092E20303
:10352000109265030E947B1B609326037093270310
:1035300080932803909329032196E2E00C944B2179
:103540000E94190E8091B902823209F011CF0CCF7E
:10355000823000F5E82FF0E0EE0FFF1FE751FC4F3F
:1035600071836083882319F08130A1F408C08091B1
:1035700069008C7F842B80936900E89A089580917C
:103580006900440F551F440F551F837F842B809380
:103590006900E99A08951F920F920FB60F921124B5
:1035A0002F933F934F935F936F937F938F939F934B
:1035B000AF93BF93EF93FF938091E9039091EA0358
:1035C000892B29F0E091E903F091EA030995FF9135
:1035D000EF91BF91AF919F918F917F916F915F918B
:1035E0004F913F912F910F900FBE0F901F90189504
:1035F0001F920F920FB60F9211242F933F934F9368
:103600005F936F937F938F939F93AF93BF93EF934A
:10361000FF938091EB039091EC03892B29F0E091CB
:10362000EB03F091EC030995FF91EF91BF91AF91FE
:103630009F918F917F916F915F914F913F912F91CA
:103640000F900FBE0F901F9018951F920F920FB6FC
:103650000F9211242F933F938F939F93AF93BF9318
:103660008091F1039091F203A091F303B091F403E0
:103670003091F5030196A11DB11D232F2D5F2D372C
:1036800020F02D570196A11DB11D2093F5038093C5
:10369000F1039093F203A093F303B093F4038091AA
:1036A000ED039091EE03A091EF03B091F00301962A
:1036B000A11DB11D8093ED039093EE03A093EF0342
:1036C000B093F003BF91AF919F918F913F912F9154
:1036D0000F900FBE0F901F9018958FB7F894209100
:1036E000F1033091F2034091F3035091F4038FBF43
:1036F000B901CA0108959FB7F8942091ED03309164
:10370000EE034091EF035091F00386B5A89B06C0ED
:103710008F3F21F02F5F3F4F4F4F5F4F9FBF542F81
:10372000432F322F2227280F311D411D511D82E0CA
:10373000220F331F441F551F8A95D1F7B901CA01C3
:103740000895EF92FF920F931F93CF93DF937B0126
:103750008C010E947B1BEB010EC00E947B1B6C1B2B
:103760007D0B685E7340C8F30894E108F108010915
:103770001109C851DC4FE114F1040105110569F785
:10378000CDB7DEB7E6E00C944721019739F0880FFA
:10379000991F880F991F02970197F1F70895789460
:1037A00084B5826084BD84B5816084BD85B5826046
:1037B00085BD85B5816085BDEEE6F0E080818160E4
:1037C0008083E1E8F0E010828081826080838081E4
:1037D00081608083E0E8F0E0808181608083E1EBBC
:1037E000F0E0808184608083E0EBF0E080818160A4
:1037F0008083EAE7F0E0808184608083808182605A
:103800008083808181608083808180688083109242
:10381000C1000895CF93DF93482F50E0CA01865628
:103820009F4FFC0134914A575F4FFA0184918823DE
:1038300069F190E0880F991FFC01E859FF4FA591AD
:10384000B491FC01EE58FF4FC591D491662351F419
:103850002FB7F8948C91932F909589238C9388811E
:1038600089230BC0623061F42FB7F8948C91932FA9
:10387000909589238C938881832B88832FBF06C0E2
:103880009FB7F8948C91832B8C939FBFDF91CF913E
:103890000895833071F0843028F48130A1F08230B3
:1038A00021F514C08630B1F08730D1F08430E9F4CE
:1038B00004C0809180008F7703C0809180008F7D4D
:1038C00080938000089584B58F7702C084B58F7D82
:1038D00084BD08958091B0008F778093B0000895E3
:1038E0008091B0008F7D8093B0000895FF920F9378
:1038F0001F93F62E482F50E0CA0182559F4FFC01BE
:103900002491CA0186569F4FFC0114914A575F4F7C
:10391000FA0104910023C9F0222319F0822F0E949A
:10392000491CE02FF0E0EE0FFF1FEE58FF4FA5916E
:10393000B4919FB7F894FF2021F48C9110958123C6
:1039400002C08C91812B8C939FBF1F910F91FF9090
:1039500008950F931F93482F50E0CA0182559F4F3F
:10396000FC012491CA0186569F4FFC0104914A57DD
:103970005F4FFA011491112319F420E030E015C0D3
:10398000222319F0822F0E94491C812F90E0880F7A
:10399000991F84589F4FFC01A591B4918C9120E010
:1039A00030E0802311F021E030E0C9011F910F9138
:1039B0000895982F8E3008F09E5097708091850260
:1039C0008295880F880F807C892B80937C00809162
:1039D0007A00806480937A0080917A0086FDFCCF23
:1039E0002091780040917900942F80E030E0282BDE
:1039F000392BC9010895A0E0B0E0E1E0FDE10C94AD
:103A000029217C016B018A01C0E0D0E00FC0D60102
:103A10006D916D01D701ED91FC910190F081E02D48
:103A2000C7010995C80FD91F015010400115110594
:103A300071F7CE01CDB7DEB7E8E00C944521DC018B
:103A4000ED91FC910190F081E02D09950895EF92A0
:103A5000FF920F931F938C016DE00E941F1D7C014C
:103A6000C8016AE00E941F1D9C012E0D3F1DC90167
:103A70001F910F91FF90EF900895EF92FF920F9397
:103A80001F937C010E941F1D8C01C7010E94271DEE
:103A90009C01200F311FC9011F910F91FF90EF90E2
:103AA0000895CF93DF93EC016115710519F420E0BF
:103AB00030E00FC0DB010D900020E9F71197A61B45
:103AC000B70BE881F9810280F381E02DAD01099502
:103AD0009C01C901DF91CF9108954F925F927F922F
:103AE0008F929F92AF92BF92CF92DF92EF92FF920E
:103AF0000F931F93DF93CF93CDB7DEB7A1970FB688
:103B0000F894DEBF0FBECDBF2C01742ECB01223046
:103B100008F42AE019A231E2C32ED12CCC0EDD1E0E
:103B2000822E9924AA24BB24672D752FA501940108
:103B30000E94E22079018A01C801B701A501940120
:103B40000E94AF20472D461B0894C108D1084A3077
:103B500010F4405D01C0495CF6014083E114F104BA
:103B60000105110521F07E2C5F2DC801DDCFC201BA
:103B7000B6010E94511DA1960FB6F894DEBF0FBE8C
:103B8000CDBFCF91DF911F910F91FF90EF90DF900C
:103B9000CF90BF90AF909F908F907F905F904F900D
:103BA0000895DC012115310541F4ED91FC9101905E
:103BB000F081E02D642F099508950E946D1D0895F0
:103BC000EF92FF920F931F939A017B0100E010E0A8
:103BD000B801A7010E94D11D1F910F91FF90EF9096
:103BE0000895EF92FF920F931F939A01E62EFF2400
:103BF00000E010E0B801A7010E94D11D1F910F91B4
:103C0000FF90EF900895A0E0B0E0E9E0FEE10C94B1
:103C10002921EC016A017B012115310541F4E8817C
:103C2000F9810190F081E02D642F09951BC02A30A5
:103C30003105B1F477FF13C06DE20E941F1D8C01A6
:103C400044275527BA014C195D096E097F09CE0139
:103C50002AE00E946D1D9C01200F311F04C02AE044
:103C60000E946D1D9C01C901CDB7DEB7E8E00C9440
:103C70004521EF92FF920F931F937B019A0100273A
:103C8000F7FC0095102FB801A7010E94031E1F9199
:103C90000F91FF90EF900895EF92FF920F931F9373
:103CA0007C010E94391E8C01C7010E94271D9C01C6
:103CB000200F311FC9011F910F91FF90EF900895C0
:103CC0000E94511D0895EF92FF920F931F937C0164
:103CD0000E94601E8C01C7010E94271D9C01200FBD
:103CE000311FC9011F910F91FF90EF900895089522
:103CF0001F920F920FB60F9211242F933F934F9361
:103D00008F939F93EF93FF938091C00082FD1DC01E
:103D10004091C60020913604309137042F5F3F4F09
:103D20002F73307080913804909139042817390727
:103D300071F0E0913604F0913704EA50FC4F408373
:103D4000309337042093360402C08091C600FF915F
:103D5000EF919F918F914F913F912F910F900FBEB7
:103D60000F901F9018951F920F920FB60F9211246B
:103D70002F933F938F939F93EF93FF9320917A0418
:103D800030917B0480917C0490917D042817390741
:103D900031F48091C1008F7D8093C10014C0E09107
:103DA0007C04F0917D04E65CFB4F208180917C04D3
:103DB00090917D0401968F73907090937D04809311
:103DC0007C042093C600FF91EF919F918F913F91CA
:103DD0002F910F900FBE0F901F901895A0E0B0E0AC
:103DE000E4EFFEE10C942521FC011382128288EE9F
:103DF00093E0A0E0B0E084839583A683B7838AEA4A
:103E000092E0918380837587648757874687318BDB
:103E1000208B138B028BF58AE48AD78AC68AB18EEF
:103E2000A08E938E828E8F85848F8889858F8989D5
:103E3000868F8A89878F8B8980A32096ECE00C94EB
:103E40004121AF92BF92DF92EF92FF920F931F93A7
:103E5000CF93DF93EC017A018B01DD24403081EEBA
:103E6000580780E0680780E0780711F0DD24D394DC
:103E700091E0A92EB12CEC89FD89DD2069F0C50106
:103E800008A002C0880F991F0A94E2F7808360E0BF
:103E900079E08DE390E005C0108260E874E88EE17F
:103EA00090E0A80197010E94E2202150304040405C
:103EB0005040569547953795279580E12030380733
:103EC00020F0DD2011F0DD24D6CFE889F989308398
:103ED000EA89FB89208319A2EE89FF89408121E0CC
:103EE00030E0C9010C8C02C0880F991F0A94E2F7D8
:103EF000482B4083EE89FF894081C9010D8C02C0A7
:103F0000880F991F0A94E2F7482B4083EE89FF89B6
:103F10004081C9010E8C02C0880F991F0A94E2F7F4
:103F2000482B4083EE89FF8980810F8C02C0220FCD
:103F3000331F0A94E2F7209528232083DF91CF9145
:103F40001F910F91FF90EF90DF90BF90AF90089579
:103F5000DC011C96ED91FC911D97E05CFF4F2191D7
:103F6000319180819181281B390B2F733070C901E9
:103F700008958EE794E00E94A81F892B11F00E94FB
:103F8000771E0895DC011C96ED91FC911D97E05C75
:103F9000FF4F20813181E054F040DF01AE5BBF4F25
:103FA0008D919C9111972817390719F42FEF3FEF46
:103FB00007C08D919C91E80FF91F8081282F30E078
:103FC000C9010895DC011C96ED91FC911D97E05C00
:103FD000FF4F20813181E054F040DF01AE5BBF4FE5
:103FE0008D919C9111972817390719F42FEF3FEF06
:103FF00010C08D919C911197E80FF91F20818D9130
:104000009C91119701968F73907011969C938E934B
:1040100030E0C9010895DC0191968C919197882335
:1040200039F05496ED91FC915597808186FFF9CF38
:1040300091961C920895CF93DF93EC01EE85FF8556
:10404000E05CFF4F20813181E054F0402F5F3F4F13
:104050002F733070DF01AE5BBF4F8D919C91119734
:1040600028173907D1F3E05CFF4F80819181E0543C
:10407000F040E80FF91F6083EE85FF85E05CFF4F9D
:1040800031832083EE89FF89208181E090E00F8CCD
:1040900002C0880F991F0A94E2F7282B208381E041
:1040A00089A3EC89FD8980818064808381E090E030
:1040B000DF91CF9108958F929F92AF92BF92CF924E
:1040C000DF92EF92FF920F931F9300D000D00F92D8
:1040D000EDB7FEB7319684E0ADB7BEB711968C93BD
:1040E00083E0818387E0828385E0838381E084832A
:1040F0008EE794E066EF73E04AE354E025EC30E0AD
:1041000004EC10E0B0ECEB2EF12CA1ECCA2ED12C7B
:10411000F2ECAF2EB12CE6EC8E2E912C0E94EE1E0E
:104120000F900F900F900F900F901F910F91FF9095
:10413000EF90DF90CF90BF90AF909F908F900895B9
:10414000CF93DF930E94CF1B0E944119C9EBDFE19F
:104150000E94C5122097E1F30E94B91FF9CF629F18
:10416000D001739FF001829FE00DF11D649FE00D6F
:10417000F11D929FF00D839FF00D749FF00D659FD0
:10418000F00D9927729FB00DE11DF91F639FB00DCF
:10419000E11DF91FBD01CF0111240895AA1BBB1B0E
:1041A00051E107C0AA1FBB1FA617B70710F0A61B37
:1041B000B70B881F991F5A95A9F780959095BC0158
:1041C000CD010895A1E21A2EAA1BBB1BFD010DC053
:1041D000AA1FBB1FEE1FFF1FA217B307E407F507B7
:1041E00020F0A21BB30BE40BF50B661F771F881F93
:1041F000991F1A9469F760957095809590959B0129
:10420000AC01BD01CF01089597FB092E05260ED004
:1042100057FD04D0D7DF0AD0001C38F450954095E4
:10422000309521953F4F4F4F5F4F0895F6F790958A
:104230008095709561957F4F8F4F9F4F08952F9276
:104240003F924F925F926F927F928F929F92AF9226
:10425000BF92CF92DF92EF92FF920F931F93CF9373
:10426000DF93CDB7DEB7CA1BDB0B0FB6F894DEBF0A
:104270000FBECDBF09942A88398848885F846E8430
:104280007D848C849B84AA84B984C884DF80EE807A
:10429000FD800C811B81AA81B981CE0FD11D0FB683
:1042A000F894DEBF0FBECDBFED010895EE0FFF1FE6
:0C42B0000590F491E02D0994F894FFCFE4
:1042BC0054582074696D656F757421005761697469
:1042CC00696E672062696E640A00476F7420706BB8
:1042DC00740A006461746120676F6F640A0052583D
:1042EC002068616E67007363616E6E6572206D6F1E
:1042FC006465004F70656E4C52536E6720525820A7
:10430C007374617274696E672000206F6E20485759
:10431C002000454550524F4D2064617461206E6FF2
:10432C00742076616C6964206F722062696E6420FF
:10433C006A756D70706572207365742C20666F726F
:10434C0063696E672062696E640A00536176656406
:10435C002062696E64206461746120746F2045452D
:10436C0050524F4D0A004920616D20736C61766587
:10437C0000456E746572696E67206E6F726D616C4C
:10438C00206D6F64650000200122012602210227A6
:10439C00032303260424052505280529052AC01214
:1043AC0000001A400AA1204EA5001B1E27522C23E8
:1043BC00308025000005400AA1204EA50020244E87
:1043CC00A52C2330004B000006400AD0009D49006C
:1043DC007B289D492C233000E1000005400A450153
:1043EC00D7DC03B81E0EBF00232E48E801008A401C
:1043FC000A6001555502AD1E20000023C88025001F
:10440C000005400AA1204EA50020244EA52C2330E7
:10441C000002000200020002000200020002000280
:10442C000002000200020002000200020002000270
:10443C008813409C080109120313000102000000BC
:10444C00100000000800200000000100000200071E
:10445C000B0C10111500000000001B20FB1CA81FEA
:06446C00E21FC21F0B203D
:107E00000F92CDB7DEB7112484B714BE81FFF1D035
:107E100082E08093C00088E18093C10086E0809377
:107E2000C20080E18093C4008EE0CDD088249924E4
:107E3000CC24C394F5E0DF2EE1E1EE2E73E0F72EC3
:107E4000B6D0082F813479F4B2D08983C2D0898129
:107E5000823811F481E005C0813811F485E001C059
:107E600083E09ED09AC0823411F484E103C085344B
:107E700019F485E0B6D091C0853561F498D0082F0B
:107E800010E095D090E0982E8824802A912A880CC2
:107E9000991C82C0863521F484E0A3D080E0E1CF34
:107EA000843609F04CC083D082D0A82E80D0B82E62
:107EB00000E011E07CD0F80181938F01AE16D1F77C
:107EC00088D0FB2DF53489F4E0E0F1E00BC0F9999E
:107ED000FECF92BC81BC0894811C911C819180BD15
:107EE000FA9AF99AEA1598F358C08B2D863409F05E
:107EF00054C0F401F7BEE89507B600FCFDCFF401CD
:107F0000A0E0B1E02C9130E011968C91119790E0B7
:107F1000982F8827822B932B12960C01C7BEE895C9
:107F20001124329681E0A038B80761F7F401D7BE7A
:107F3000E89507B600FCFDCFE7BEE8952EC0843774
:107F4000F1F435D034D0182F32D0B82E42D0FB2DDA
:107F5000F63421F4F40105914F010CC0FB2DF534EA
:107F600049F4F999FECF92BC81BC0894811C911C04
:107F7000F89A00B5802F14D0115049F70EC08537FC
:107F800039F427D08EE10CD085E90AD08FE069CF93
:107F9000813511F488E017D01CD080E101D050CF9A
:107FA0009091C00095FFFCCF8093C600089580910A
:107FB000C00087FFFCCF8091C00084FD01C0A89560
:107FC0008091C6000895E0E6F0E098E19083808318
:107FD0000895EDDF803219F088E0F5DFFFCF84E10E
:107FE000DFCF1F93182FE3DF1150E9F7F2DF1F9166
:0E7FF0000895282E80E0E7DFEE27FF27099492
:027FFE0001057B
:0400000300007E007B
:00000001FF
